:040000006F00503C01
:10000400000000000000000000010020AA050020FC
:10001400A9BDF9F300010020000000000000000069
:10002400000100200001002000000000000000008A
:100034008806002000000000BC060020000000002C
:100044002806002028060020280600202806002074
:1000540028060020000100202806002000000000DF
:100064002806002028060020280600202806002054
:100074002806002028060020280600202806002044
:100084002806002028060020280600202806002034
:100094002806002028060020280600202806002024
:1000A40000010020C2030020000100200001002004
:1000B40000010020000100200001002000000000D9
:1000C40000010020000100200001002000010020A8
:1000D4000001002000010020000100200001002098
:1000E4000001002000010020000100200001002088
:1000F4000001002000010020000100200001002078
:100104006F000000B7170040984B411113670701B7
:1001140098CB982B1377E70F98AB130780087337A6
:100124000780137787083AC60F100000130770057D
:100134002380E704130780FA2380E7040F100000EC
:10014400B847B70600069506558FB8C703C7B70466
:100154001377F70DA385E704B82713672701B8A71A
:10016400130750149AA7372700408346578093F605
:10017400F60EA302D7808946A303D78003C7E704FA
:100184001377C70F136717002387E70403C7F70222
:1001940013672700A387E702982B1367170098AB10
:1001A40023800704B247F3A707800F100000410122
:1001B4008280EFF03FF513054027970500009385F3
:1001C400650B171600001306E69F63FCC500832227
:1001D400050023A055001305450093854500E3E879
:1001E400C5FE174500E01305E552971500009385F9
:1001F400659D1386818163FCC5008322050023A0CD
:1002040055001305450093854500E3E8C5FE1385B5
:100214008181973500009385A5CB6378B5002320B1
:10022400050013054500E36CB5FE9302500273907C
:1002340002BC9302300073904280930200007390DA
:1002440012BCB7220000938202807390023097029E
:100254000000938222DB93E23200739052309712B3
:1002640000E0938202AA73901234730020300000DD
:10027400011122CC8D4505453714004026CA4AC8D1
:100284004EC606CE1309840B971000E0E78060B8D1
:1002940085448549232039011305401F972000E038
:1002A400E780001C9307C40A84C31305A00F97209A
:1002B40000E0E780E01AF9BF31712ED332D536D78A
:1002C4002A86541193050008080806CF22CD3AD98E
:1002D4003EDB42DD46DF36C61384C181973000E041
:1002E400E78040C50840FD55972000E0E780C08ABC
:1002F4000C08174500E01305A516973000E0E780C9
:10030400C0A80840814601468145971000E0E78077
:10031400C03CFA406A4429618280411122C406C665
:10032400174400E013040414228579371305401F91
:10033400972000E0E780C012C5BF01110D4681453A
:10034400054522CC06CE26CA4AC84EC613848181EE
:10035400971000E0E780203108C029C9854505656C
:10036400971000E0E780E0AA89450565971000E052
:10037400E78060BAB7E700E03707020023A0E71080
:100384000549974400E093846410974900E09389F9
:10039400690E0840FD55971000E0E780E07F631583
:1003A40025014E85113FF5B72685EDBF6244F24025
:1003B400D2444249B249174500E01305A50E056130
:1003C400E5BDB717004083D7C7090111056722CCE3
:1003D40006CE33C40708F98F99CF6C0003A5818139
:1003E400971000E0E7800052B24791C7B7E700E0FA
:1003F400116723A0E720B7170040F240239E870827
:10040400624405618280B7F70700DC53411123A6DB
:10041400F182B7170040984B1367070198CB982BCC
:100424001377E70F98AB13078008733707801377A8
:1004340087083AC60F100000130770052380E704ED
:10044400130780FA2380E7040F1000001307000C41
:100454006315E5029A271367070C9AA7B71700409C
:10046400982B1367170098AB23800704B247F3A7B0
:1004740007800F10000041018280B8279376052081
:10048400ADCA118B29E303C7E70403C6E704137756
:10049400F70F136636002387C704B0271366460098
:1004A400B0A792278E273346060893E5050C8EA73E
:1004B400A5470100FD1793F7F70FE5FFB7170040B5
:1004C40092A72387E70493770510DDC3371700400D
:1004D4003C2793E707013CA79377F50199EFB727EA
:1004E400004003C7578013670701A382E7801D47B5
:1004F4000DA013672700B8A7F9B725476366F7046B
:10050400B727004003C757801377F70EA382E7800D
:100514000547A383E78033450508B71700401367F1
:10052400050C9AA78AA7B5CE03C7570483C65704F8
:10053400418B858A558F1DF3B82B418B05D3B82782
:100544001377D70FB8A719BF9377050199EBB7278E
:10055400004003C757801377F70EA382E78009474B
:100564004DBFB727004003C757801377F70EB5BFB9
:100574009377850181EFB727004003C7578013772E
:10058400F70EA382E7801307100561B7B727004071
:1005940003C757801377F70EA382E780130770050C
:1005A4008DBFB8271377B70F71BF4111814601463C
:1005B40081451145CD2C13078008F337078093F745
:1005C40087083EC40F100000B717004013067005DB
:1005D4002380C704930680FA2380D7040F100000F9
:1005E400FD55CEB723800704A245F3A505800F105F
:1005F400000073370780137787083AC60F1000008E
:100604002380C7042380D7040F10000003C76704A6
:10061400136717002383E70423800704B247F3A773
:1006240007800F10000001A0F325203493952500C6
:1006340017050000130505A33305B50003250500C0
:10064400F32210BC13F31200631C03027310013471
:1006540003A1018173E010BC73600430E70005005E
:100664007370043013000000130000001300000036
:1006740073F010BC130000007321003473002030A9
:10068400E700050073002030972000E0E78080B485
:1006940011C5B7E700E0116723A0E720B7F700E032
:1006A40023A207007300203073700430010001009E
:1006B400010082807360043082800000197106C2D8
:1006C40016C41AC61EC822CA26CC2ACE2ED032D2AE
:1006D40036D43AD63ED842DA46DC4ADECEC0D2C25E
:1006E400D6C4DAC6DEC8E2CAE6CCEACEEED0F2D28E
:1006F400F6D4FAD6FED892DA9305000273A04580A8
:1007040083A2418823A02200F32510342EC0EF00D9
:10071400400503A3418803210300824273901234ED
:100724009240A2423243C2435244E244724582554B
:100734001256A2563257C2575258E2587259864935
:10074400164AA64A364BC64B564CE64C764D865D49
:10075400165EA65E365FC65F56520961730020308E
:10076400000083A7C18489C7854723A0F1868280BE
:1007740023A001861385C1861C4197260000938619
:10078400E65F5148338707033386E6000C4285C58C
:100794004C4221073697CC414CC26394E500D841C2
:1007A40058C251473387E702BA96D842584723A222
:1007B400E1881CC1828085EB411106C67370043048
:1007C4000100010001008565174600E01306C6DE3E
:1007D400938575BF174500E0130505D8972000E001
:1007E400E780A05A01A0FD1771BF230304801547B9
:1007F4002303E48001002302A480828083076480B1
:10080400E3CE07FE23030480828083076480E3CE63
:1008140007FE03454480828083076480E3CE07FE9D
:100824002302A4808280411126C44AC24EC006C657
:100834001377F50BAD47AA892E8995446306F70013
:1008440019456537653F8D444E854537FD59FD147F
:1008540063983401B240A244124982494101828022
:10086400135509011375F50F453F2209CDB7011141
:1008740026CC06CEB704080051371545BD3771376D
:1008840069372AC6A53F32459377150089EB13656E
:1008940015001375F50FF240E24405618280FD14E2
:1008A400E9FC0145CDBF3971B7F7070006DE26DC48
:1008B4004ADA4ED852D656D45AD25ED062CE03AB60
:1008C40047027D57B7E700E083AA070022C603AAC0
:1008D400470023A0E71823A2E718B71B004093079B
:1008E40070052380FB04930780FA2380FB0483C7ED
:1008F4004B041147AA8993E7070E2382FB0437248C
:1009040000401305F00F2303E4802E8C3289B68453
:10091400E93DED35938779FF93F7F70F0947137B8B
:10092400FB006362F712A147370708006307FB0067
:10093400B70707003E9C378707007955637EEC02B2
:10094400B3878401636AF702A9476398F90689E4C7
:1009540081446D3526850DA0E2850945E9350509F3
:100964000345F9FFFD14050C453D81C49377FC0F45
:10097400FDF7F53D69FD7D55B71700401307700578
:100984002380E704130780FA2380E70403C747049E
:10099400418B2382E704F250B7E700E023A057110C
:1009A40023A24711E25432445259C259325AA25A2C
:1009B400125B825B724C21618280A547639AF906BF
:1009C400A1478569631DFB029387F9FFB3869700EE
:1009D400B374FC00B69493C7F7FFFD8C33FC870116
:1009E400416B856B9387F9FFB3F7870199E363FF45
:1009F400340193D94900C147E3E637FF91BF930718
:100A0400F00FE9B78567C169FD17C9B71305800DF4
:100A140063886901130500026384790113051008D2
:100A2400E2851135A93521D94E9CB3843441C1B72F
:100A3400E2852D45CD3BCA94E30C99F00509F133C9
:100A4400A30FA9FED5BF9387F9FF93F7F70F636F41
:100A5400F70AA1476319FB06B70708003E9C83C742
:100A64005B043707070093F7070299E3378707000A
:100A7400B70708003E977955E370ECF0B3079C0084
:100A8400E36CF7EE8947639AF9048980D549E381D9
:100A940004ECE2850945413B11090327C9FF91474D
:100AA4002320E48003076480E34E07FE230334819C
:100AB400FD17EDFBFD14110C81C49377FC0FE9FFC6
:100AC4007D3371F54DBD83C75B043707070093F78A
:100AD4000702D5F33787070079BF8547E384F9F226
:100AE400E2852D4589339389F4FFE38304E6313BA2
:100AF40093F7390091EB83260480032709009307B9
:100B04004900E398E6E43E89CE84F1BFB547639695
:100B1400F9001305900BD13925BDB1471305B00A6F
:100B2400E38BF9FE99476394F904A1476315FB002D
:100B3400B70708003E9CE2852D45F53181440D4BF5
:100B4400A149E13163966401832704802320F900DD
:100B54008504E39834FF8327048013172C0163551D
:100B640007002312F900EDB32322F900D5B39D4702
:100B74006399F90281451305B0047531BD442320FE
:100B8400090023220900FD59493193F77400CA97DB
:100B940003C70700FD14398D2380A700E39634FFB3
:100BA40045BB91476399F900130560063D39B93196
:100BB400130590098DB7E38D09D8F15459BB000092
:100BC400971100209381C18517F10120130141433E
:100BD4001305400097F5FF1F9385854217F6FF1F05
:100BE4001306066963FCC5008322050023A0550093
:100BF4001305450093854500E3E8C5FE17F5FF1F7F
:100C04001305255B6700050003A14188024182406A
:100C14003243C2435244E244724582551256A256AC
:100C24003257C2575258E25872598649164AA64A50
:100C3400364BC64B564CE64C764D865D165EA65E2C
:100C4400365FC65FD652A10273900230A242096198
:100C540082800100F322003093F272FF13038018A4
:100C64001203B3E26200711523205500130585FABF
:100C740010C12115232005008142638702007115EC
:100C840023200500FD12D5BF71150CC182802A8373
:100C940009CA83830500230073007D1605038505B7
:100CA4006DFA82802A8311C62300B3007D160503E2
:100CB40065FE828015C22A8385466367B500FD56AA
:100CC4001307F6FF3A93BA95838305002300730054
:100CD4007D163693B6956DFA8280411106C6B71714
:100CE4000040116723ACE70AC1450545592C8D45E1
:100CF4001165212AB240410159AE4111114506C680
:100D040022C465281305503497F0FF1FE780A06FB5
:100D1400296585457D15D52885457D55852A753FE9
:100D24001735000013054579EF20A0190545EF009C
:100D3400F03923AEA18001E9173500001305457889
:100D4400EF20201801A093870182394781461306BA
:100D54000010973500009385E57717F5FF1F1305FD
:100D6400C55DEF10E01B938741821547814613064A
:100D74000010973500009385657617F5FF1F13055E
:100D8400C559EF10E01993878182154781461306F0
:100D94000010973500009385E57417F5FF1F1305C0
:100DA400254DEF10E017EF104038173400001304FE
:100DB400E4732285EF20E010EDBF3717004083472E
:100DC400E70412054111BD8BC98F93F7F70F930602
:100DD4008008F3B6068093F6860836C60F10000026
:100DE400930670052300D704930680FA2300D704E2
:100DF4000F1000002307F70423000704B247F3A7EA
:100E040007800F10000041018280914763ECB70412
:100E1400973700009387076FB3C5F52098413E9735
:100E2400B71700409387470B028794433717004056
:100E3400B3F6A64094C39306070B9C42B3F7A740AE
:100E440019A8944337170040B3F6A64094C39306F9
:100E5400070B9C42C98F9CC29307070A98433377B8
:100E6400A74098C38280944337170040C98ED9B7EE
:100E740098433377A74098C3B71700409387070A6E
:100E84009843498FF9BF9843498FF5B7914763EC6D
:100E9400B7049737000093872768B3C5F5209841B6
:100EA4003E97B71700409387470D0287944337173F
:100EB4000040B3F6A64094C39306070D9C42B3F7D3
:100EC400A74019A8944337170040B3F6A64094C32B
:100ED4009306070D9C42C98F9CC29307070C984345
:100EE4003377A74098C38280944337170040C98E54
:100EF400D9B798433377A74098C3B717004093876F
:100F0400070C9843498FF9BF9843498FF5B7894730
:100F140033470508638BF50463E2B7021346F7FF12
:100F24009DE9B717004083D64709F18E239AD70865
:100F34009387C70A9443C98E94C321A08D47638CB9
:100F4400F502B7170040239EE70883D60709558F9B
:100F54002398E7088280B717004083D64709F18EAB
:100F6400239AD7089387870AF1B7B717004083D627
:100F74004709D98E65BFB717004083D64709D98E74
:100F8400C5B719C5371700401E2FCD8F1EAF8280FD
:100F9400B71700409A2FB375B7408EAF8280B7174A
:100FA40000409A279306000C1377070C630AD704B2
:100FB4009A27137707100DC79A279E277D8B09EB75
:100FC40093F70720B1C33755E801130505808280E4
:100FD40037C59812FD8B130505E03345F502828071
:100FE4009A279E2713770720FD8B11C73755E801F1
:100FF40013050580DDB73725F40013050540F1BF5F
:101004002165130505D082803725F40013050540BA
:1010140082803285814737370040A14663C3A700E9
:1010240082803037E30FD6FE3386F5001022850721
:1010340010A7EDB797060020938686BEAA8788423C
:1010440017270020130787E8AA9763E9E7000A87B0
:10105400130707FC6364F7009CC282807D5582807D
:10106400411122C406C62A841D3F2947B307E5025D
:10107400B2408D83B3D7870222449507B3D7E702E2
:1010840037370040B3C707085EA741018280716506
:1010940041111305052006C6E137B7370040130791
:1010A40070F8B8A30D47B8B31307000498B3054705
:1010B400F8A7B24041018280938741843E879C43D4
:1010C400E3EEA7FE50435441B305C700631AB500CD
:1010D400B29654C33306D7006394C7023A8529A055
:1010E4003306D500639FC70003A601846386C70047
:1010F400D043B296904354C110C16303A70008C300
:1011040082801CC1DDBF011122CC06CE26CA4AC88A
:101114004EC62A84EF10000A138601841C42B9E7E4
:1011240017070020130707BB9376F700896799CA4E
:10113400170700201307F7BA419B972700209387CE
:1011440067B9998FBA97C117C19B23A4018423A2BD
:10115400E18423A2070023A00700B386E7401CC252
:101164001CC354C323ACD18223AED18219C4937758
:10117400F4001387F7FD637D8700EF1080190149A0
:10118400F2406244D244B2494A85424905618280B0
:1011940013050402B306F540E351D0FE9389C183DD
:1011A40083A40900E3EBD4FC1387418400434C403F
:1011B40063F6D50003280400631608041042E30E06
:1011C40086FA1040898F03290700AE9710C31307CE
:1011D4000002637FF7023305D4001377F50015C7C7
:1011E400737004300100010001001736000013067B
:1011F400E6339305C00D173500001305A535EF1030
:10120400503801A0228742845DB75CC154C06D355B
:101214005840938681839042B387E44023A0F90029
:1012240063F3C7009CC21317F72958C0138741837F
:101234001C4323200400410985071CC3EF10600DE3
:101244009377F90095DF7370043001000100010009
:10125400173600001306862D9305C01117350000BC
:101264001305452FEF10F03101A051C9832745FF25
:10127400411122C406C62A8463C407027370043071
:10128400010001000100173600001306262A930509
:10129400F012173500001305E52BEF10902E01A076
:1012A400032705FF1DC37370043001000100010012
:1012B4001736000013068627930500131735000020
:1012C40013054529EF10F02B01A09397F749232A22
:1012D400F5FEEF00306E1387C1831443832744FF68
:1012E400130504FFB6971CC3C13B138701831C433A
:1012F4002244B24085071CC341016F1080018280E3
:10130400B7E700E039472388E70417F7FF1F1307FF
:10131400E73A13671700B8D33147A388E70417F7F0
:10132400FF1F1307673613671700F8D3130700F876
:101334002387E74093860710116690C22386E7400F
:10134400B7F700E0796723A407001307F77798CB72
:10135400056798C23D4798C38280011106CE02C634
:10136400F32750303EC6B2470D478D8B6384E702A6
:1013740073700430010001000100173600001306E9
:10138400A61F93053007173500001305A51CEF10A1
:10139400501F01A097F70120938787C6BD8B9DC37B
:1013A40073700430010001000100173600001306B9
:1013B400A61C93058007173500001305A519EF1027
:1013C400501C01A0353FEFF03F84F2400145056118
:1013D4008280930785007D575CC118C55CC51CC914
:1013E4002320050082802328050082809441FD5734
:1013F40013078500639DF6001C49D843D8C10CC768
:101404009CC5CCC31C4188C985071CC18280BA878E
:1014140058431043E3FDC6FECDB7544118451C495B
:1014240098C654C3D4436393A600D8C398432328CF
:1014340005007D1798C388438280411122C42A8401
:1014440006C697F0FF1FE7802026005C97F0FF1F79
:10145400E7804026B24013351400224441018280C3
:1014640041114AC03289304126C2045D22C406C6F5
:101474002A8405E21C4195EB0845EF1080412324A2
:101484000400850404DCB240224492440249410130
:101494008280631109024841EFF06FFF5C403840DD
:1014A400BA9718445CC063F4E7000145D9BF1C40F7
:1014B4005CC0E5BF4845EFF08FFD38405C44B3069F
:1014C400E040998F18405CC463F5E7001C44B6976C
:1014D4005CC489470145E316F9FAC5D4FD1455B730
:1014E400AA87B0432E8501CED84794473297D8C7F0
:1014F4006364D7009843D8C7CC476FF04FF9828014
:10150400411122C42A8426C24AC006C697F0FF1F8E
:10151400E78080198344540413094402939444607B
:1015240063419004FD57A302F40497F0FF1FE78082
:10153400601897F0FF1FE7802017834444041309C1
:10154400040193944460634A9002FD572302F40417
:101554002244B24092440249410117F3FF1F67003D
:1015640063155C50E1D34A85EF10A00A19C1EF104E
:101574006025FD149394446065B71C48F9D74A85E7
:10158400EF10200919C1EF10E023FD149394446077
:101594005DBF411106C622C426C21DE1737004302A
:1015A40001000100010017360000130666FF9305D1
:1015B400E012173500001305E5F9EF10807C01A057
:1015C4005C5D2A84BDCB3841B3B7E702BDE7AE8486
:1015D40097F0FF1FE780400D34405C5C1840232CDB
:1015E4000402B387F60258C03306F700958F3E977E
:1015F400FD572302F40410C458C4A302F4049DE468
:101604001C4899CB13050401EF10A00011C5B7E7DE
:1016140000E0116723A0E72097F0FF1FE78080090F
:10162400B2402244924405454101828013050401DD
:101634004D3313054402713BC5B773700430010088
:101644000100010017360000130686F593053016D5
:1016540017350000130505F0EF10A07201A0411129
:1016640006C622C426C24AC039C1B337B5022A8984
:10167400AE8495EF3305B502930770FB63E9A702C7
:101684001305850449342A8401CDAA8799C0930798
:1016940085041CC0232E240324C085452285D53D02
:1016A400B2402285224492440249410182807370EF
:1016B400043001000100010017360000130646EE55
:1016C4009305401E173500001305C5E8EF10606B45
:1016D40001A0397106DE22DC26DA4AD84ED652D46D
:1016E40056D25AD032C61DE1737004300100010095
:1016F4000100173600001306A6EA9305C034173517
:101704000000130525E5EF10C06701A02A842E8987
:10171400B6848DE53C419DC3737004300100010023
:101724000100173600001306A6E79305D0341735D9
:101734000000130525E2EF10C06401A089476398F7
:10174400F402585C85476304F702737004300100A7
:101754000100010017360000130686E49305E03407
:1017640017350000130505DFEF10A06101A0EF108D
:10177400E00519E1B247A1EB97F0FF1FE780C0F243
:10178400185C5C5C6373F7062686CA852285C939B2
:101794005C5089C713054402EF00B06711C5B7E771
:1017A40000E0116723A0E72097F0FF1FE78080F097
:1017B4000545F2506254D2544259B259225A925AAF
:1017C400025B21618280737004300100010001001A
:1017D400173600001306C6DC9305103517350000D4
:1017E400130545D7EF10E05901A08947E38EF4F8BB
:1017F4008147FD59130B040137EA00E0916A71A097
:1018040081E72808EF00506F97F0FF1FE78080EA18
:10181400EF00501A97F0FF1FE78000E98347440464
:101824009397476063943701230204048347540465
:101834009397476063943701A302040497F0FF1F52
:10184400E78040E76C002808EF00F06B3DE997F073
:10185400FF1FE78060E5185C5C5C6310F70497F099
:10186400FF1FE78020E5B2455A85EF00B04F22857F
:101874004139EF00102A39C197F0FF1FE780C0E219
:101884001C5C585CE3E2E7F08547324735FB97F090
:10189400FF1FE78020E2014529BF97F0FF1FE78083
:1018A40060E12285B139EF00D02697F0FF1FE78071
:1018B400A0DF185C5C5CE379F7FCF9B523205A21BE
:1018C400EDB722853539EF00D024F1B741112A86CE
:1018D4008145054522C406C659332A8419C92324DF
:1018E4000500232005002326050081460146814585
:1018F400CD33B2402285224441018280411106C683
:1019040022C426C24AC01DE17370043001000100E4
:101914000100173600001306A6C89305904C17352E
:101924000000130525C3EF10C04501A03C412A84E3
:101934009DC37370043001000100010017360000DC
:10194400130606C69305D04C17350000130585C051
:10195400EF10204301A01C412E898DE71C459DC337
:1019640073700430010001000100173600001306F3
:1019740026C39305204D173500001305A5BDEF10B0
:10198400404001A01C5C585C63FEE7068344540499
:1019940085071CDCFD57939444606395F4025C5006
:1019A40099CB13054402EF00D04611C56305090025
:1019B40085472320F9000545B24022449244024958
:1019C40041018280EF003000E3F7A4FE9307F007A3
:1019D4006394F402737004300100010001001736AF
:1019E40000001306E6BB93051055173500001305D8
:1019F40065B6EF10003901A0850493944460A302F6
:101A0400940455BF01454DBF397106DE22DC26DA48
:101A14004AD84ED632C61DE173700430010001006D
:101A24000100173600001306A6B79305B056173504
:101A34000000130525B2EF10C03401A02A842E89BA
:101A44008DE53C419DC37370043001000100010029
:101A5400173600001306C6B49305F0561735000078
:101A6400130545AFEF10E03101A0EF0030560DE54E
:101A7400B2479DC3737004300100010001001736A2
:101A840000001306E6B1930540571735000013050F
:101A940065ACEF10002F01A097F0FF1FE780C0C0D6
:101AA400045C95CCCA852285FD141D3C04DC1C48CD
:101AB40099CB13050401EF00D03511C5B7E700E059
:101AC400116723A0E72097F0FF1FE780A0BE05451C
:101AD400F2506254D2544259B25921618280B247C1
:101AE40099E797F0FF1FE780E0BC0145D5B72808C8
:101AF400EF009040FD5997F0FF1FE780A0BBEF0077
:101B0400606B97F0FF1FE78020BA834744049397E4
:101B14004760639437012302040483475404939772
:101B2400476063943701A302040497F0FF1FE78022
:101B340060B86C002808EF00103D31E12285EFF019
:101B4400DF8F0DC9B24513054402EF00B021228591
:101B5400453AEF00007C11E5B7E700E0116723A0E8
:101B6400E72097F0FF1FE78020B4045C85FCB247B0
:101B7400D9F385BF22856932EF00A079DDB72285CC
:101B84004132EF0000792285EFF03F8B79D9B1BF64
:101B9400397106DE22DC26DA4AD84ED652D456D221
:101BA4005AD02EC61DE173700430010001000100FB
:101BB400173600001306C69E9305D05F1735000044
:101BC40013054599EF10E01B01A03C412A849DC3F5
:101BD4007370043001000100010017360000130681
:101BE400269C93051060173500001305A596EF1089
:101BF400401901A0EF00903DAA842DC10149814400
:101C0400FD59130A4402B7EA00E0116B97F0FF1F75
:101C1400E78080A91C5CA5CBFD171CDC1C4081E778
:101C2400EF00706108C41C4899CB13050401EF0050
:101C3400501E11C5B7E700E0116723A0E72097F015
:101C4400FF1FE78020A70545F2506254D254425941
:101C5400B259225A925A025B21618280B2470149E9
:101C6400C5D3737004300100010001001736000071
:101C74001306069393056060173500001305858DE0
:101C8400EF10201001A0B24799E797F0FF1FE780FB
:101C940060A2014555BF81E42808EF00F02597F0C4
:101CA400FF1FE78020A1392397F0FF1FE780C09F23
:101CB40083474404939747606394370123020404E1
:101CC400834754049397476063943701A302040441
:101CD40097F0FF1FE780009E6C002808EF00B022F9
:101CE40029E52285EFF06FF505CD1C4089EF97F0CB
:101CF400FF1FE780609B0844EF00902E2A8997F02D
:101D0400FF1FE780209BB2455285EF00B005228576
:101D1400EFF00FFFFD2B19E123A06A218544FDB5E7
:101D24002285EFF0EFFDF523D5BF2285EFF04FFDBF
:101D3400CD232285EFF06FF075D1E30C09F497F011
:101D4400FF1FE78060964C5089C51C58BD459C43D5
:101D54009D8D0844EF0050400DBF15E5411106C6A6
:101D6400737004300100010001008565173600001E
:101D740013060683938585AD172500001305857D1D
:101D8400EF10200001A08DCD17170020130787F452
:101D9400814781463A882146832847006397A800F3
:101DA400B3E706218CC3C8C321A891E783280700A1
:101DB40063930800BA8785062107E39FC6FCFDF3F9
:101DC4008280411122C426C24AC02A8406C6AE8437
:101DD400328997F0FF1FE780208D834744047D57A5
:101DE400939747606394E7002302040483475404F1
:101DF4007D57939747606394E700A302040497F028
:101E0400FF1FE780208B1C5C99E74A86A685130593
:101E14004402EF00A07922852244B2409244024950
:101E240041016FF0EFED011122CC1384418826CAE1
:101E34004EC6AA8483A901871C4008404AC806CE1E
:101E4400A388070411052E89EFF02FDDFD57639059
:101E5400F404630E0902971700209387A7EB14403C
:101E6400D84398C610471440D0C61440910654C2B3
:101E74001440910614C718405CCB9843050798C3D7
:101E8400F2406244D2444249B249056182801C4016
:101E9400CE94C4C363FE340103A5C1870C406244DD
:101EA400F240D2444249B249910505616FF00FD422
:101EB40003A501880C409105EFF04FD3938741852A
:101EC4009843E3FFE4FA84C365BF9387418803A77B
:101ED400C1869C43C85719EF05E51717002003274F
:101EE400A7E9854763EFE70003A5418583A7018739
:101EF4001D8D828011E59717002083A7E7E7828074
:101F040001458280138701881C439443938741854C
:101F140081E67D5798C38280184358471843DDBF34
:101F2400797126D2931426005AC82A8B26854ECE60
:101F340052CC56CA5EC606D622D44AD02E8AB68B56
:101F4400BA89BE8AEFF02F9C09ED7D55B250225418
:101F540092540259F249624AD24A424BB24B456109
:101F640082802A8913054005EFF0EF992A84630AD9
:101F7400051A130640058145EFE0DFD22328240328
:101F840063020A020147C146B307EA0083870700D8
:101F94003306E400230AF60281C70507E316D7FED9
:101FA400A3010404B94763F43703737004300100D8
:101FB40001000100172600001306C65F93052039AF
:101FC4001725000013050559EF00B05B01A0130AA3
:101FD400440052852326340323223405EFF0AFC096
:101FE40013058401EFF02FC0BD47F114B3873741C7
:101FF400CA9400C81CCC40D05E86DA8513F504FF71
:10200400EFE05FC508C063840A0023A08A0097E05C
:10201400FF1FE7806069938741879843138941884C
:1020240097140020938444D5050798C30327090017
:10203400631D070C23208900984385476317F7061F
:10204400A689971A0020938AEAE54E85D109EFF014
:102054004FB8E39C3AFF171500201305A5D0EFF005
:102064004FB7171500201305A5CEEFF08FB617153F
:1020740000201305A5CCEFF0CFB5171500201305EC
:10208400A5CAEFF00FB5171500201305A5C8EFF08A
:102094004FB4971700209387E7CC23A0F1889717B4
:1020A40000209387E7CA23AEF186138781851C43FA
:1020B40085071CC31387C1865C54144363F3F6007D
:1020C4001CC35147B387E702A697D843144718C4E3
:1020D40054C423A246012324470198435CC805073E
:1020E40098C397E0FF1FE780E05C83A7818681CFD8
:1020F40083270900D8575C546377F700B7E700E0FB
:10210400116723A0E720054591B503A781865C5498
:1021140049FF032709005857E3E9E7F8232089001A
:1021240069B74A85EFF06F940DB541119387018526
:102134000147814613060008972500009385C5488A
:10214400170500001305453722C406C60544C93BDC
:10215400631C8502EF00903D6318850273700430A0
:10216400010001000100FD5723AAF18423A4A186E4
:1021740023A80186EFF06F9EB240224497F7FF1F19
:1021840083A747AA41018280FD57E317F5FE7370C8
:1021940004300100010001008565172600001306C4
:1021A400664193852581172500001305A53AEF00A4
:1021B400503D01A01387C1841C4385071CC3828042
:1021C40003A50187828003A54187828083A7C184F8
:1021D4006398071241119387018722C4804306C67E
:1021E400050480C329E4938701889843184305C7ED
:1021F400737004300100010001008565172600009A
:102204001306463B938575AB1725000013058534EB
:10221400EF00303701A01387C1879443104390C364
:1022240014C31387C1851C4385071CC3E139138676
:1022340041851C4201456379F40083A70186E1EBE3
:10224400B240224441018280938801881383C1866D
:10225400971E0020938E4EB2514F938F418851A800
:1022640083A70800DC47DC47D8436374E40018C242
:10227400E9B78C47D447D84B1388470094C5CCC2E0
:102284004C436393050154C3144323AA0700FD166A
:1022940014C398570DC3CC4F9453032E470094C5D1
:1022A400CCC2938587016313BE0054C3144323A493
:1022B4000702FD1614C3D457032703006374D70021
:1022C4002320D3003387E60376974C4303AE85007F
:1022D4008CC723A6C70123220E0123A40501D8CB52
:1022E4001C4385071CC383A70F00DC5763F3D70087
:1022F400054583A708009C43A5F7FD571CC235BFBD
:10230400138741861C43014585071CC3828005450C
:1023140005BF011122CC1384C1841C4006CE26CAF9
:102324004AC885E773700430010001000100856527
:1023340017260000130606289385558817250000E4
:1023440013054521EF00F02301A097E0FF1FE7806C
:10235400A0351C40FD171CC01C4091CF01452AC666
:1023640097E0FF1FE7800035F24062443245D244D3
:1023740042490561828083A74187EDD381471715C0
:1023840000201305A59B1388C1861713002013038F
:10239400A39E514E938E4188138F0186854FBDA80D
:1023A4005C45DC479857D04F94534C4314C6D0C275
:1023B400138687016393C50054C3144323A40702FF
:1023C400FD1614C39047D447D84B9385470014C6D1
:1023D400D0C250436313B60054C31443FD1614C350
:1023E40003270800D4576374D7002320D800338709
:1023F400C6031A9750438328860090C723A6170163
:1024040023A2B8000CC61043D8CB050610C303A7FB
:102414000E00585763E4E6002320FF01184149F3F6
:1024240099C3EFF03FAE03A4418601CC93840186A7
:102434000549693B19C123A024017D147DF823A219
:10244400018683A70186E38B07F0B7E700E01167F5
:1024540023A0E720054521B719E5B7E700E0116798
:1024640023A0E7208280011106CE83A7C1849DC3E7
:1024740073700430010001000100172600001306E8
:1024840066139305C051172500001305A50CEF0032
:10249400500F01A02AC6393B32458145EFF0BF9861
:1024A4008D3D11E5B7E700E0116723A0E720F24076
:1024B40005618280011122CC4AC84EC652C456C25C
:1024C4005AC006CE26CA13848187171A0020130A1D
:1024D400AA85138941878549938A4185138B01878E
:1024E4001C409DEFEFF07F9EE3FCA9FEE13103A7C2
:1024F4000A0083270B006373F7067370043001002E
:10250400010001008565172600001306A60A9385BD
:10251400A5DB172500001305E503EF00900601A0D5
:1025240097E0FF1FE78040188327CA00C44713853C
:102534004400EFE09FEE83270900FD172320F900F4
:102544001C40FD171CC097E0FF1FE780A0168858A9
:10255400EFE0BFD12685EFE05FD159B7EFF0FF96EA
:102564004D3BBDBF411106C622C405E5737004305E
:10257400010001000100856517260000130686038B
:102584009385F5C0172500001305C5FCEF00607F97
:1025940001A02E8483A54188E105EFE03FE5228573
:1025A4002244B240854541016FF0FF87AA8715E5B3
:1025B400411106C6737004300100010001008565F5
:1025C40017260000130606FF938555C4172500003F
:1025D400130545F8EF00E07A01A013874188D4433E
:1025E4002E85B285104303A8860054CE10432320C1
:1025F4000603104361062322C800104318436106F2
:1026040090C61CD79843050798C391C17D556FF0B8
:102614009F815C45411122C4C04706C605E473701E
:10262400043001000100010085651726000013062F
:1026340066F8938555C7172500001305A5F1EF002B
:10264400407401A01C54544C1850D04398C654C331
:10265400930684016313D600D8C398432324040249
:102664007D1798C383A7C184ADEB5C4814445844D8
:10267400D04398C654C3930644006313D600D8C30A
:1026840098437D1798C31387C1865C5410436373C2
:10269400F6001CC351473387E7029707002093874E
:1026A400A76DBA97D843104718C450C454C214C76E
:1026B40098435CC8050798C3EFF0DF8483A741887B
:1026C4005854DC57014563F6E700854723A0F1869B
:1026D4000545B24022444101828097070020938738
:1026E400E765D843104758CC10D054C214C7984358
:1026F4001CD4050798C3D9B783A7C1851CC183A778
:1027040001875CC18280011106CE22CC1DE1737069
:10271400043001000100010085651726000013063E
:1027240066E9938505CF172500001305A5E2912DD1
:1027340001A02E849DE173700430010001000100AA
:102744008565172600001306E6E6938515CF172541
:102754000000130525E0352501A02AC697E0FF1FD8
:10276400E78080F49387418883A6018790433245AC
:1027740003461605584119CE9C43A3880704054512
:102784002AC697E0FF1FE780E0F2F2406244324538
:10279400056182801C407D566384C7020C4103A6F8
:1027A400C1856387C50063E5E60023200400C1BF3B
:1027B4003386E640E37BF6FE958FBA971CC02D3F27
:1027C40001457DBF854723A0F186828083A781864A
:1027D400054591C703A5C1841335150006058280FC
:1027E4005DC501114AC813894188032709005C5556
:1027F40022CC585706CE26CA4EC62A8463F2E7086E
:10280400184D634807000327090054573D47158FA7
:1028140018CD5147B387E7025848970400209384A2
:10282400A455A6976319F704930944004E85EFE075
:10283400DFBE832709001387C1861443DC575CD4A9
:1028440063F3F6001CC35147B387E702A697D84346
:10285400144718C454C423A23601232437019843CF
:102864005CC8050798C30545F2406244D244424916
:10287400B2490561828083270900DC575CD4E5B73F
:10288400832709006841DC573335F500F1BF014562
:10289400828009E9014582800145B2402244924484
:1028A40041018280411122C406C626C283A7418801
:1028B4002A846384A70273700430010001000100BC
:1028C4008565172600001306E6CE93859504172523
:1028D4000000130525C8752101A0BC479DE3737052
:1028E400043001000100010085651726000013066D
:1028F40066CC9385A504172500001305A5C55121B1
:1029040001A054557841FD173CC5E387E6F8C9F7A3
:10291400930445002685EFE05FB07C403D471D8F62
:1029240018CC1387C18614435CD463F3F6001CC32C
:102934005147B387E702170700201307E74305450C
:10294400BA97D843144718C454C4C4C204C798439C
:102954005CC8050798C391B771CD3845411122C4AD
:1029640006C626C24AC02A841DE3737004300100DF
:10297400010001008565172600001306A6C3938590
:102984009509172500001305E5BCE52E01A07C413F
:10299400B3F5F50A5C556389B70885466316D7080D
:1029A40003A741886314A702737004300100010077
:1029B40001008565172600001306C6BF9385450BE5
:1029C40017250000130505B96D2E01A0184D4CD52F
:1029D400634507003D470D8F18CD5147B387E70284
:1029E40058489704002093842439A697631EF7025D
:1029F400130944004A85EFE05FA21387C1865C5443
:102A0400144363F3F6001CC35147B387E702A69748
:102A1400D843144718C454C423A2260123242701ED
:102A240098435CC8050798C3B240224492440249C3
:102A340041018280828093874188984309C79443E7
:102A4400B8460507B8C688438280411106C64CC102
:102A540008C9AA876361B602184D158E05456379C6
:102A6400E6009385470003A54189EFE03F980145BF
:102A7400B240410182806375D6000545E3FAD5FE74
:102A84009385470003A58189CDB7411122C426C28D
:102A94004AC006C62A84AE8432890C4CA6864A866D
:102AA400A69522855D3719E5B24022449244024935
:102AB400410182801C4C2285BE941C508297F1BF38
:102AC40083A78189DC47011122CCC04726CAAA8486
:102AD4001305440006CE2EC6EFE03F94834744021C
:102AE400324613F7470019CBA6852285793F1C503F
:102AF40022856244F240D24405618287F99B230215
:102B0400F402F5B7011122CC26CA4AC84EC606CE35
:102B1400AA8413898188EFF0AFEA832709002A8405
:102B2400938981896362F502814723208900F240F9
:102B3400228562449CC04249D244B24905618280E4
:102B4400DC47FD558843AD3F83A7090098436DFBDF
:102B54001387418914431CC3854723A0D900F1B7C7
:102B64005D71A6C2CAC04EDE52DC86C6A2C4938979
:102B7400818993840189138A4189172900001309E3
:102B8400A9A683A709000546804301C4DC47014682
:102B9400804332C6EFF00FE20810AD378257AA85A2
:102BA400B5EB324629E6636985042AC6EFF06FF671
:102BB400B24522853137884001460C10EFE0DFE44E
:102BC40069D18257225563CA070422545C48A9EF8D
:102BD40068080D3F825721472A86FD17E36DF7FCED
:102BE400B3C727219843834744024A970287832720
:102BF4000A009043133616008840B305B440EFF042
:102C04004F9CEFF00FF145F9B7E700E0116723A0FF
:102C1400E72055B7EFF0EFEF79BF9257B25582979F
:102C24008257E3CA07F855B713054400EFE0EFFEF7
:102C340045B793E717002302F4020C4C92562AC6B8
:102C44002285B695193525D983474402324613F7B0
:102C5400470011CB1C4C92552285BE953D351C5026
:102C64002285829789BFF99B2302F402CDBF93E7A3
:102C740017002302F40292550CCC95E173700430D2
:102C84000100010001001726000013066694930555
:102C9400E035172500001305E58BE52001A0AA8681
:102CA400AA9522855D3301BF13F7270009E7228522
:102CB400EFE0AFDB09B7F99B2302F402EDBD41114C
:102CC40022C406C61384018997E0FF1FE780C09DD4
:102CD4001C40B1E7170500201305051EEFE06FEF58
:102CE400170500201305051CEFE0AFEE9707002041
:102CF4009387871C23ACF1880146970700209387AC
:102D0400671AC145114523AAF188EFE05F9508C011
:102D140019C5972500009385658FEFF00F84224431
:102D2400B240410117E3FF1F6700C398411106C673
:102D3400793783A7018995E373700430010001009A
:102D44000100172600001306A68893059011172585
:102D5400000013052580352001A09387C1883947D9
:102D6400814613060008972500009385A58A170558
:102D74000000130525DFEFF0AF9A5DDDB24041019D
:102D840082805D7122D406D62A842EDA32DC36DEC5
:102D9400BAC0BEC2C2C4C6C603A5818011C51C4D3B
:102DA40081E72AC6D92332450C455418228636CEEB
:102DB400EF102014B250225461618280011126CA9E
:102DC40006CE22CC4AC84EC652C4AA8419E11C4578
:102DD40002901C4D2E89B5E3492B9C4C8044A5C31D
:102DE4009727000093878787631EF404C0407C50B4
:102DF400858B81EB5E2493F7072081E7284CEF0055
:102E0400406E5E24A18B99C31C48D5E3A285268518
:102E1400DD2251CDFD547C50858B99E75E2493F7D8
:102E2400072099E3284C7D2DF24062444249B2497F
:102E3400224A2685D24405618280004555B72685FD
:102E44002D2379BF971700009387477F6314F400FD
:102E5400804471BF971700009387477CE319F4F807
:102E6400C04471B71CC4050963C807021C4013871A
:102E7400170018C08CA31C4483450900FD17FDF1FD
:102E84001CC463D907022286A94526857D20FD57E7
:102E9400E302F5F8A94441B7184C63C4E700E3978B
:102EA40045FD228626855128E31735FDA5B7FD5932
:102EB400294AD1B71C401387170018C0294798A383
:102EC400D1BFAA8503A58180D5BD1971A2DCA6DA7C
:102ED40086DECAD8AA843284635C06009307B008ED
:102EE4001CC17D55F6506654D654465909618280FA
:102EF40093078020FC822EC42ECC36868147BA8666
:102F040019C09307F4FF7D592C0026853EC83ECE98
:102F1400231B2101EF00101A635525019307B00804
:102F24009CC069D0A247238007006DBF3687B28654
:102F34002E86AA8503A5818049BF011122CC26CA09
:102F44004AC806CE4EC6AA842E89328401C51C4DB9
:102F540091E3212997170000938747706317F402C0
:102F6400C0401C4C1CC45E24A18B99C31C4895EF23
:102F7400A2852685492015C97D59F2406244D24470
:102F8400B2494A85424905618280971700009387B8
:102F9400E76A6314F4008044E9B797170000938745
:102FA400E767E310F4FCC0446DBF1C480840937904
:102FB400F90F1379F90F1D8D5C486346F500A2855E
:102FC4002685912C55F91C440505FD171CC41C408D
:102FD4001387170018C0238037015C486388A70053
:102FE4005E24858BD9DBA947E319F9F8A2852685E8
:102FF4001D2441D551B7411122C426C24AC006C678
:1030040083A481802A892E8489C49C4C99E32685D3
:10301400A92E97170000938767646313F402C040D6
:103024008317C40013F7870025E713F707010DEB97
:1030340025472320E90093E707045EA47D5571A08A
:10304400971700009387875F6314F4008044C9BF17
:10305400971700009387875CE314F4FCC044C9B756
:10306400918B9DC34C5889C9930744046384F5002C
:103074004A858D23232A04025E242322040093F725
:10308400B7FD5EA41C481CC05E2493E787005EA4C1
:103094001C4899EB5E241307002093F707286385E7
:1030A400E700A2854A8569298317C40013F717002E
:1030B4001DC35848232404003307E04018CC1848A3
:1030C400014501E713F707083DF7B2402244924453
:1030D40002494101828013F72700814611E35448D5
:1030E40014C4F1BF8397C500011122CC26CA06CEB1
:1030F4004AC84EC613F78700AA842E8479E3D841C0
:103104006345E000B8416356E008585459C303A925
:10311400040023A004000C5093D7C748A9CB7048DF
:103124005E24918B99C75C401D8E5C5899C33C40CA
:103134001D8E5C540C50814626858297FD57630C86
:10314400F5041C480567232204001CC05E24F98F83
:1031540091C368C84C5823A0240185CD9307440427
:103164006384F5002685BD21232A04021DA001469F
:10317400854626850297FD572A86E313F5FA9C4077
:10318400C5D375476385E70059476395E70623A0D0
:1031940024010145B5A098408317C40001CFF5462A
:1031A4006305D700D9466319D7041C4823220400B9
:1031B4001CC04DB718482322040093D7C74818C031
:1031C40041BF83A90501E38609FC03A905008D8B92
:1031D40023A0350133093941014791E3D84918C483
:1031E400E35920FB1C540C50CA864E8626858297D0
:1031F400634FA0008317C40093E707045EA47D55C2
:10320400F2406244D2444249B24905618280AA999B
:103214003309A940F1B79C49411106C622C426C20C
:1032240081EB8144B240224426859244410182804C
:10323400AA842E8401C51C4D91E3052A971700002A
:103244009387C741631CF402C0408317C400F1DBB9
:103254007850058B11E793F7072099E3284C512404
:103264002685A28541357C50AA84858BC5FF5E24C2
:1032740093F70720C5FB284CB5246DB797170000BA
:103284009387C73B6314F4008044C1B797170000C9
:103294009387C738E31BF4FAC04445BF411122C4E5
:1032A40006C62A844EA572A5232005002322050004
:1032B400232405002322050623280500232A0500CC
:1032C400232C0500214681451305C505EFD09F9D9C
:1032D40097170000938727F05CD097170000938717
:1032E40027F21CD4971700009387E7F55CD497174F
:1032F4000000938727F8B24000D01CD82244410133
:10330400828097050000938545F1BDA2411126C234
:10331400930780069384F5FFB384F4024AC02E8990
:1033240022C406C69385440765262A8401CD23203A
:10333400050023222501310508C41386840681452E
:10334400EFD05F96B2402285224492440249410163
:1033540082801385018A71A21385018A61A2138573
:10336400418A41A21385418AB5AA411122C406C6E5
:103374002A84F5371C4C89C72244B2404101DDB789
:1033840097070000938727F81CD4232404042326DA
:1033940004042328040483A7418163948700854798
:1033A4001CCC22853D2048C02285252008C42285C6
:1033B4000D2048C4484001469145CD350844054692
:1033C400A545E93D48440946C945C93D85471CCC46
:1033D40065B7411126C24AC006C622C42A89953F50
:1033E40083A441819C4C99E32685413793848404CA
:1033F4008044DC40FD1763D607009C40BDC3844075
:10340400C5BF0317C40039EBC17785075CC4130536
:10341400840523220406E920813721462320040061
:10342400232404002322040023280400232A040064
:10343400232C040081451305C405EFD0BF86232A3D
:103444000402232C04022324040423260404B2408B
:103454002285224492440249410182801304840655
:1034640051BF91454A855D3588C02A8449F9ED35B7
:10347400B1472320F900E1BF797122D44AD04ECE5E
:1034840052CC5AC85EC606D626D256CA2A892E8A75
:10349400130485048149054BFD5B0444832A4400DD
:1034A400FD1A63D00A0200406DF8B25022549254BF
:1034B4000259624AD24A424BB24B4E85F2494561A7
:1034C4008280DE24637BFB008397E40063877701BB
:1034D400A6854A85029AB3E9A90093848406C9B7EC
:1034E4008280828082805971A2D42E848395E500E3
:1034F400A6D2CAD086D6B284368963D205025E24A7
:1035040093F7070895EB13070040B6502654232081
:10351400F90098C0065996540145656182803000CF
:10352400EF00905AE34D05FC3247BD67F98F797778
:10353400BA9793B71700C1BF814713070004F1B7C7
:10354400DE25797122D406D626D24AD04ECE898B76
:103554002E8491CF930774041CC01CC885475CC893
:10356400B250225492540259F24945618280740047
:103574003000AA848D3FA2492A892685CE85892ACE
:1035840019E98317C40013F7072079FBF19B93E72C
:1035940027005EA4C1B7970700009387C7D69CD4C1
:1035A4005E2408C008C893E707085EA4B247232A2C
:1035B400340181CF8315E4002685EF00705311C5D3
:1035C4005E24F19B93E717005EA45E2433E5270194
:1035D4004AA479B7C5C183A7C5FF011122CC06CE81
:1035E4001384C5FF63D307003E942AC6EF00D05668
:1035F4001387C18A1C43324589EB2322040000C38C
:103604006244F24005616F00B055637DF4001040E0
:10361400B306C4006396D7009443DC43B29614C047
:103624005CC0F1BF3E87DC4399C3E37DF4FE1443E1
:103634003306D700631F86001040B29614C33306C6
:10364400D700E39FC7FA9043DC43B29614C35CC32C
:1036540045BF6375C400B1471CC15DB71040B306D4
:10366400C4006396D7009443DC43B29614C05CC094
:1036740040C379B7828041114AC01389818A832764
:10368400090022C426C206C6AA842E8491E7814575
:10369400EF00B0312320A900A2852685EF00F03089
:1036A4007D59631A25017D54B240228522449244F7
:1036B400024941018280130435007198E30685FEB6
:1036C400B305A4402685EF00502EE31F25FDE1BF7E
:1036D400011126CA93843500F1984AC8A104B14760
:1036E40006CE22CC4EC62A89B3F4F40A63C404007D
:1036F40063FDB400B1472320F9000145F240624460
:10370400D2444249B24905618280EF00F044938972
:10371400C18A83A709003E8439E4A6854A85A13F6E
:10372400FD572A846319F50A03A40900A287D1EB83
:103734008329040081454A85A299EF0010276395E7
:10374400A9081C408D044A859D8CF198B147A104B9
:10375400B3F4F40AA6850537FD576307F5061C4044
:10376400A6971CC015A01440858E63C906042D4776
:10377400637ED70204C0330794006397870223A0B3
:10378400E9005C4014C35CC34A85EF00703D130537
:10379400B4009307440061993307F540E300F5F65C
:1037A4003A94898F1CC099BFD8C3E1BF5840639530
:1037B400870023A0E900C9BFD8C3F9B7A287404056
:1037C400A1BF3E84DC43A5B7B1472320F9004A8555
:1037D400EF0010391DB704C145BF01114AC803A940
:1037E400850022CC4EC652C456C206CE26CA5AC042
:1037F40003AA05002E84B28AB68963E42607839758
:10380400C50013F7074821CF58488D448C49B38429
:10381400E4020947330ABA4093F707402A8BB3C43A
:10382400E402138716005297B3F4E40ABDC3A685D5
:1038340045352A893DC50C485286EFD04FC55E24D4
:1038440093F7F7B793E707085EA42328240144C835
:103854005299B38444412320240104C44E8963F360
:1038640029014E8908404A86D685EFD0AFC41C444E
:103874000145B38727411CC41C40CA971CC0F240B1
:103884006244D2444249B249224A924A024B0561F7
:1038940082802686EF00502D2A8945F90C485A85E6
:1038A400153BB1472320FB005E247D5593E70704B5
:1038B4005EA4F1B7DE25357122CD26CB4AC952C5A7
:1038C40006CF4EC756C35AC1DEDEE2DC93F70708C3
:1038D4002A8A2E89B28436849DCF9C498DEF930524
:1038E4000004FD332320A9002328A9000DE1B147DA
:1038F4002320FA007D55FA406A44DA444A49BA4919
:103904002A4A9A4A0A4BF65B665C0D6182809307E9
:103914000004232AF90093070002A304F102930789
:10392400000302D22305F10222C6930B5002971A18
:103934000000938AAAD4294B26841C2099C3639837
:103944007709330C9440630D9400E2862686CA8579
:1039540052856135FD576307F5189257E2973ED2B9
:103964001C2063810718FD579304140002C802CE7B
:103974003ECA02CCA309010482D48C201546568584
:10398400EF00101CC2471384140021E513F707014C
:1039940009C713070002A309E10413F7870009C745
:1039A4001307B002A309E10494201307A00263895A
:1039B400E602F24726848146254618209305140022
:1039C400130707FD6372E60685C63ECE15A00504FF
:1039D400ADB733055541B397A728A2843EC871BF3C
:1039E400324793064700184336C6634807023ACE67
:1039F40018209307E002631CF70418309307A00211
:103A0400631AF702B2470904138747009C433AC676
:103A14007D57B3E7E70A3ECA1DA83307E04093E7A2
:103A240027003ACE3EC8E9B7B38767032E8485469C
:103A3400BA9761B7050402CA814681472546182012
:103A440093051400130707FD6374E606E9F60C20DA
:103A54000D46171500001305E5C2EF00700E11CDD9
:103A640097170000938707C21D8DC24713070004F0
:103A74003317A700D98F05043EC80C201946171523
:103A84000000130565C0930414002304B102EF0081
:103A9400300B2DC19307000095E74247B2471377D7
:103AA400071009CF91073EC69257CE973ED269B50B
:103AB400B38767032E848546BA9751B79D07E19B68
:103AC400A107D5B7780097060000938646D14A86A9
:103AD4000C08528597000000E7000000FD57AA89F2
:103AE400E314F5FC8357C90093F70704E39407E054
:103AF400125511B5780097060000938646CE4A8683
:103B04000C0852853922D9BF797156CA9C49BA8AA0
:103B1400984522D44AD04ECE52CC06D626D25AC884
:103B24005EC6B3E7E70A1CC203C73504AA892E841C
:103B34003289368A19C385071CC21C4093F70702D1
:103B440091C78327090089072320F9000440998835
:103B540091E8130B9401FD5B5C4403270900998FE2
:103B640063CCF40483473404B336F0001C4093F769
:103B74000702A5EB13063404D2854E85829AFD57BD
:103B84006303F5041C4011478144998B6399E70052
:103B94008327090044449D8C8147B3E4F40A1C4400
:103BA40018486354F700998FBE94014969047D5BFA
:103BB40063982405014509A885465A86D2854E8511
:103BC400829A631E75017D55B25022549254025953
:103BD400F249624AD24A424BB24B45618280850423
:103BE400A5BF3307D40013060003A301C70403478A
:103BF400540493871600A2978906A381E7049DBF06
:103C040085462286D2854E85829AE30E65FB050998
:103C140045B7797122D44AD04ECE52CC06D626D29C
:103C240056CA5AC803C88501930780072A892E8477
:103C3400B289368A63E20703930720069386350424
:103C440063E10703630B081C930780051716000044
:103C5400130606A46307F81493042404230104053B
:103C640015A89307D8F993F7F70F5546E366F6FEC0
:103C740017160000130646A4B3C7C7209C43B29787
:103C840082871C4393842504938647009C4314C372
:103C94002381F504854765A290411C4313750608EA
:103CA4009385470029C19C430CC3584063DE071227
:103CB4009305D002A301B40418C4635E0702B307DA
:103CC400F040171600001306A69C2948B68433F763
:103CD4000703FD143297182398A03E87B3D7070330
:103CE400E37707FF85A09C43137506040CC355DDD9
:103CF400939757605DBF6D9A10C0D1B790411C4334
:103D0400137506089385470001C50CC39C4331A075
:103D1400137606040CC37DDA9E231307F0061716E8
:103D240000001306E696631FE80A2148A301040471
:103D3400584018C4E34C07F80C40ED990CC0D9F76F
:103D4400B68449F7A147631EF8001C40858B91CBCC
:103D540058401C4863C7E70093070003A38FF4FE91
:103D6400FD14858E14C85287CE867000A2854A85BC
:103D7400613BFD5A6319550D7D55B250225492543E
:103D84000259F249624AD24A424B456182809C41BF
:103D940093E707029CC11308800717160000130657
:103DA4006690A30204050C401C4313F80508138510
:103DB40047006305080008C39C4339A013F80504B1
:103DC40008C3E30B08FE9E2313F7150001C793E510
:103DD40005020CC099C3414891BF18401377F7FD01
:103DE40018C0D5BF294899B7171600001306468A8C
:103DF40029483DBF90411C43CC49137806081385DC
:103E040047006306080008C39C438CC339A008C359
:103E1400137606049C4375DA8EA323280400B68423
:103E240099B71C43D04181459386470014C384430A
:103E34002685392301C5B30795405CC05C401CC886
:103E4400A30104040DB714482686CE854A85029A38
:103E5400E30455F31C40898B85E74844B247336536
:103E6400F50A21BF85465686CE854A85029AE30522
:103E740065F185045C443247998FE3C5F4FEF1BFD4
:103E84008144930A94017D5BF5B71C46FD171CC65B
:103E940063DA0700184E63C5E700A9476394F50089
:103EA4006FF0AF891C422E851387170018C28CA3AC
:103EB4008280011122CC26CA4AC84EC652C406CEFC
:103EC4002A89AE893284B304D6007D5A63149400DF
:103ED400014501A80C204E864A85453F0504E31799
:103EE40045FFF2406244D2444249B249224A056144
:103EF4008280357122CD26CB4AC94EC706CF52C522
:103F040056C35AC1DEDEE2DCAA892E843289B68425
:103F140009C51C4D99E3EFF04FC59707000093873F
:103F2400E7736318F40403A449007C50858B81EB88
:103F34005E2493F7072081E7284CEFF08FDA5E24A4
:103F4400A18B99C31C48A5E3A2854E85EFF0AF8AE7
:103F540039C97C50858BA1C37D55FA406A44DA4443
:103F64004A49BA492A4A9A4A0A4BF65B665C0D6189
:103F74008280970700009387676C6315F40003A49D
:103F8400890065B79707000093874769E31FF4F832
:103F940003A4C90059BF5E2493F70720D5FF284C1A
:103FA400EFF04FD455BF93070002A304F102930727
:103FB400000302D22305F10226C6930B5002970A8E
:103FC4000000938AAA6B294BCA849C2099C36399E5
:103FD4007709338C2441638D2401E2864A86A285C5
:103FE4004E85C13DFD576306F5189257E2973ED2C0
:103FF4009C2063800718FD571389140002C802CE61
:104004003ECA02CCA309010482D4834509001546A3
:1040140056853D26C2479304190029E513F7070185
:1040240009C713070002A309E10413F7870009C7AE
:104034001307B002A309E104834609001307A00291
:104044006389E602F247CA8481462546982093850F
:104054001400130707FD6372E60685C63ECE15A05D
:104064008504A5B733055541B397A72826893EC8CB
:1040740069BF324793064700184336C663480702B0
:104084003ACE98209307E002631CF7049830930714
:10409400A002631AF702B2478904138747009C43BE
:1040A4003AC67D57B3E7E70A3ECA1DA83307E04086
:1040B40093E727003ACE3EC8E9B7B3876703AE84D7
:1040C4008546BA9761B7850402CA81468147254669
:1040D400982093851400130707FD6372E606E9F63A
:1040E4008C200D46170500001305C559912C11CDE0
:1040F40097070000938707591D8DC24713070004D3
:104104003317A700D98F85043EC88C20194617059C
:10411400000013056557138914002304B1020D240C
:1041240035C99307000095E74247B2471377071054
:1041340009CF91073EC69257D2973ED271B5B38745
:104144006703AE848546BA9761B79D07E19BA107D3
:10415400D5B77800970600009386E6D522860C082A
:104164004E8597000000E7000000FD572A8AE314FB
:10417400F5FC7C50858B81EB5E2493F7072081E767
:10418400284CEFF02FB65E2493F70704E39607DC80
:104194001255E1B37800970600009386C6D12286B3
:1041A4000C084E85EFF0FFA6C9B7411122C42A843A
:1041B4002E8523A8018A06C6EFC0DFE7FD576316E4
:1041C400F50083A7018B91C31CC0B2402244410176
:1041D4008280411122C42E848395E50006C6012401
:1041E400634905007C48AA977CC8B2402244410137
:1041F40082805E249397C7485EA4C5BFDE25011163
:1042040022CC26CA4AC84EC606CE93F70710AA8403
:104214002E843289B68991C78395E5008946014683
:10422400DD285E248315E400F2409397C7485EA41A
:104234006244CE864A86B24942492685D244056103
:104244001DA8411122C42E848395E50006C6E120F1
:104254007D575E246319E5009397C7485EA4B24076
:104264002244410182809397C72868C85EA4C5BFD1
:104274008395E5003DA0411122C42A842E85B28590
:10428400368623A8018A06C6EFC0BFD8FD57631639
:10429400F50083A7018B91C31CC0B24022444101A5
:1042A4008280411122C42A842E8523A8018A06C64D
:1042B400B522FD576316F50083A7018B91C31CC07B
:1042C400B240224441018280411122C42A842E85B5
:1042D400B28523A8018A06C6812AFD576316F50014
:1042E40083A7018B91C31CC0B24022444101828048
:1042F400411122C42A842E8523A8018A06C61D2AB8
:10430400FD576316F50083A7018B91C31CC0B2400F
:10431400224441018280411122C42A842E85B2851F
:10432400368623A8018A06C6212AFD576316F5009E
:1043340083A7018B91C31CC0B240224441018280F7
:1043440093F5F50F2A966314C500014582801C215C
:10435400E38EB7FE0505C5BF1385C1896FF06F985D
:104364001385C1896FF00F98011126CA06CE22CC9D
:104374004AC84EC652C4B28499E96244F240D24457
:104384004249B249224AB28505616FF06FB409EE21
:10439400EFF04FA40144F24022856244D2444249E2
:1043A400B249224A056182802A8A2E84B1282A8948
:1043B4006366950093571500E3EF97FCA685528535
:1043C400EFF00FB1AA8979D5A28533D6240BEFC0BB
:1043D4001F8CA2855285EFF0EF9F4E846DBF411173
:1043E40022C42A842E85B285368623A8018A06C66D
:1043F400B128FD576316F50083A7018B91C31CC038
:10440400B24022444101828083A7C5FF1385C7FFC0
:1044140063D50700AA959C413E9582809307800549
:1044240023A8F18A7D5582809307800523A8F18A09
:104434007D5582809307800523A8F18A01458280F7
:104444009307800523A8F18A7D5582809307800510
:1044540023A8F18A7D558280257300007461736BF3
:10446400322072756E6E696E67210A007461736B17
:1044740033204750494F2077616B65207570210ABE
:10448400000000007461736B332073656D206765F1
:1044940074206661696C65640A0000007461736B62
:1044A400332073656D20696E6974206661696C657B
:1044B400640A000073746172742E00007072696E75
:1044C400744D75746578206572726F720000000017
:1044D4007461736B330000007461736B320000000D
:1044E4007461736B3100000073686F756C646E27C0
:1044F400742072756E2061742068657265212100D4
:104504002AC9FFFF42C9FFFF66C9FFFF70C9FFFF49
:1045140086C9FFFF98C9FFFFB0C9FFFFD4C9FFFFD9
:10452400DEC9FFFFF4C9FFFF2E2E2F4672656552C8
:10453400544F532F706F727461626C652F4D656DAB
:104544004D616E672F686561705F342E63000000F3
:10455400657272206174206C696E65202564206F19
:10456400662066696C6520222573222E200D0A20A0
:10457400000000002E2E2F4672656552544F532FB3
:10458400706F727461626C652F4743432F524953B5
:10459400432D562F706F72742E6300002E2E2F46FB
:1045A40072656552544F532F71756575652E63009E
:1045B4002E2E2F4672656552544F532F7461736BC0
:1045C400732E630049444C45000000002E2E2F46F4
:1045D40072656552544F532F74696D6572732E63FF
:1045E400000000004EE6FFFF4EE6FFFFD2E6FFFFAD
:1045F4008AE6FFFFC4E6FFFF4EE6FFFF4EE6FFFF3D
:10460400D2E6FFFF8AE6FFFF546D725100000000FE
:10461400546D722053766300000000000000000017
:104624000000000000000000000000000000000086
:104634000000000000000000000000000000000076
:104644000000000000000000000000000000000066
:104654000000000000000000000000000000000056
:104664000000000000000000000000000000000046
:104674000000000000000000232D302B200000006B
:10468400686C4C006566674546470000303132333C
:10469400343536373839414243444546000000003A
:1046A40030313233343536373839616263646566A4
:1046B40000000000CEF5FFFFE4F5FFFFA4F5FFFFC7
:1046C400A4F5FFFFA4F5FFFFA4F5FFFFE4F5FFFF4A
:1046D400A4F5FFFFA4F5FFFFA4F5FFFFA4F5FFFF7A
:1046E40040F7FFFF48F6FFFFDAF6FFFFA4F5FFFFF0
:1046F400A4F5FFFF6EF7FFFFA4F5FFFF48F6FFFFE9
:0C470400A4F5FFFFA4F5FFFFE2F6FFFFA5
:10471000000000005C4600003C4600001C46000013
:104720000000000000000000000000000000000089
:104730000000000000000000000000000000000079
:104740000000000000000000000000000000000069
:104750000000000000000000000000000000000059
:104760000000000000000000000000000000000049
:10477000CC2E00200E000000C00B00200000000026
:0847800000000220C00B002024
:00000001FF
